:020000040000FA
:0400000019202F286C
:08000800F000030EF100831269
:10001000031383130408F2000A08F3000B1973207A
:1000200073088A0072088400710E8300F00E700E4F
:100030000900830103018500BB00FF3086008316A1
:10004000F3308500003086008312831691308100E2
:10005000831207309F0081018B018B1608008F20CF
:100060009D20FF30A300A501B801FF30B900BA0000
:100070008101A2018B175820230203193B28240871
:10008000A3002514B8010A302402031C4F28263E81
:1000900084000008BA002708B90025103B2823086F
:1000A000263E84000008BA00FF30B90025103B2826
:1000B0000508A4000301051A6828A41C0138241CA3
:1000C0000238A41F0438241F0838013EA400080089
:1000D000A418013824180238A41B0438241B08383B
:1000E000013EA40008000B11A20A25180800782878
:1000F000FF308600F3303B05B81D0438B8190838C6
:10010000BB00850038080739303E84003908B8192B
:100110003A0800048600B80A0F30B80508002630F7
:1001200084000030A0000A30A1002008AB2080002D
:10013000A00A840AA10B9528080030308400FE3004
:10014000A0000830A100200880000314A00D840A3C
:10015000A10BA328080083169B001C141A08831205
:02016000080095
:084000000000030003000000B2
:02400E00703F01
:10420000C000F900A400B000990092008200F800FC
:04421000800090009A
:00000001FF
